:1000000033C04CC063C717CB49C048C047C046C0C7
:1000100045C0D2C643C00FCA11C8FECA9DC751CC45
:100020007BC73CC03BC07068583858380004080C87
:100030000100090802060004030201000002010099
:1000400001000000010000000000000000010204A7
:100050000604020000020608000000000000B8B814
:10006000B8B8B8B80000000011241FBECFE5D4E036
:10007000DEBFCDBF10E0A0E6B0E0E2E1FDE102C0EE
:1000800005900D92A63EB107D9F711E0A6EEB0E0BB
:1000900001C01D92A737B107E1F74FC6B1CF9698BF
:1000A000A898C098109256011092550181E0809353
:1000B000110180931501089583B7836083BF88B7CA
:1000C000816088BF89B7816089BF87EC82BF08954E
:1000D0008EB587608EBD08956B9A80910B018FB9A4
:1000E000779BFECF8FB1C19AC198A99A089580914C
:1000F00013018823A1F080910B01877880930B0175
:10010000E9E2F0E09491892B80930B01E5DF87E031
:10011000809324018091FA00837C8C6117C08091C8
:1001200012018823A9F080910B01877880930B013D
:10013000E8E2F0E09491892B80930B01CDDF8BE016
:10014000809324018091FA00837C8C628093FA0072
:10015000C3DF089540914F01342FE7E2F1E024E03E
:1001600081913823215027FFFBCF21E09091450159
:10017000892F822321F4832F822309F0922B220FCF
:10018000B9F79093450180915001892B80935001DC
:10019000342FE7E2F1E024E08191382B215027FF52
:1001A000FBCF21E090914501892F822331F0832FED
:1001B000822319F4822F80959823220FA9F7909318
:1001C000450190912C01E92FFF27E95DFE4F408307
:1001D0008091500186958695869580934601892F5A
:1001E0008F5F80932C01853010F020932C010895AF
:1001F0000895AB98AB9A37E020E083B3992744E0A9
:10020000969587954A95E1F781709070032E02C00C
:10021000880F991F0A94E2F7282BAD98AD9A3150B8
:10022000383058F3209520934F010895CF93C09113
:100230001501CC2309F06CC0C0930B0180910E0115
:10024000811155DFC0931801C0936C00C0936B00FF
:10025000C0931701C0931601C093150181E08093EC
:10026000100180936900C0930F0110925401109205
:10027000530110924E0110924D01109226011092DE
:100280002501969A80910E01882371F08091460194
:100290008B3051F480910D01882331F0B09B02C066
:1002A000A898C098A89A05C0989B02C0A898C09822
:1002B000C09A1092240110924C0110924B0110929E
:1002C0003A01109239018091390190913A0190934D
:1002D00038018093370180913701909138019093D4
:1002E00036018093350180913501909136019093CC
:1002F00034018093330110923B01EEDE80E0EDEE9D
:10030000F0E0873009F010828F5F31968E30C8F3AD
:10031000CF91089590E08350883008F491E0892FC0
:10032000992708956B9890E0A92FBB27FD01E05B0A
:10033000FF4F84918FB9779BFECF8FB1A95BBE4FE2
:100340008C918FB9779BFECF8FB1C298C29A9F5F75
:10035000943050F3809147018093F50080914801DB
:100360008093F600809149018093F70080914A01C3
:100370008093F80008951092140180910E01882353
:1003800081F090910C01992331F081E0809312016A
:1003900010921301089581E080931301909312014C
:1003A0000895809313018093120108950895809118
:1003B0001F018093E90080915901E82FFF27909158
:1003C0002201843018F4E95BFE4F02C0EB5BFE4F64
:1003D00080818093EA009093EB008091E600809307
:1003E000EC000895CF9380915A019927AA2797FD91
:1003F000A095BA2FBC01CD01F0DBDC01CB012DECC7
:100400003CEC4CE45DE3BC01CD0131DCDC01CB0113
:10041000BC01CD01C5DBDC01CB01C82F8091ED0013
:1004200090910B01853748F48091E60081608093BC
:10043000E6009F7790930B01B7C08091E6008E7F16
:100440008093E6009068977890930B018091590112
:10045000E82FFF27EA5DFF4F8491982B90930B01C3
:100460003BDE8091E60083FF48C08091E600877FF5
:100470008093E6008091E60084608093E60080919E
:1004800057019927807C90708038910521F48091E4
:1004900059018A5F16C0809157019927807C90701E
:1004A000803C910519F4809159010BC0809157014E
:1004B0009927807C90708034910529F480915901AE
:1004C000845F80932E0180912E01E82FFF27E55055
:1004D000FF4F108210922D0180915901843008F055
:1004E000825080932F0180912F01E82FFF27E95B35
:1004F000FE4F108217DF109222018091E60082FFEA
:1005000053C0F09122016F2F7727E0915A012E2FCF
:1005100033274C2F5527C901841B950B6817790782
:1005200074F0240F351F261737074CF08091E60032
:100530008B7F8093E6008091E600826021C08F2F40
:1005400099274E0F511D8417950724F08091E600DE
:10055000886011C0809130018F5F809330018230BC
:1005600018F190912D019F5F90932D019E3F58F0BF
:100570008091E60080618093E6008091E6008B7FA9
:100580008093E60011C080912E01E82FFF27E550EF
:10059000FF4F908380912F01E82FFF27E95BFE4FEB
:1005A0009083C0DE10923001CF9108959F92AF9258
:1005B000BF92CF92DF92EF92FF920F931F93CF9350
:1005C000DF93CC249C2CC0E0D0E0E0913101E330FB
:1005D00011F414E005C0E43011F413E001C01E2F43
:1005E00080910B01887F812B80930B0175DD70E07A
:1005F000369B369A80911A018823E1F324B185B1A4
:100600009927982F88273327822B932BC80FD91F20
:1006100010921A017F5F783058F3E12FFF27E45ED4
:10062000FE4F15E0D695C7951A95E1F7C0838091E6
:1006300031018630E9F4809146018F31C9F480910F
:1006400057019927807C90708038910581F08091C6
:1006500057019927807C9070803C910541F08091F2
:1006600057019927807C90708034910509F4BADE97
:1006700080911F018093ED0010913101153009F038
:1006800041C08B3140F080913201843020F48F5F83
:100690008093320106C08091ED008A3110F41092EF
:1006A0003201809132018430D0F090911C019695F6
:1006B000969580911D0186958695890F912D911DA6
:1006C00020911E0126952695820F911D20912001D3
:1006D00026952695820F911D95958795982E809148
:1006E00057019927807C90708038910531F42DE076
:1006F000291540F0AEE09A2E05C049E0491510F0EA
:10070000FAE09F2EC091ED00C031C8F08091460103
:1007100001DE882339F080911C018093EF008091E5
:100720001D0102C08093EF008093F00080911E01B4
:100730008093F100809120018093EE0008C0109218
:10074000EF001092F0001092F1001092EE008091F4
:1007500021018093F200809123018093F300809126
:100760000B01D0904601CB3110F0806801C08F772B
:1007700080930B018FE1D81609F4DBC0809114013E
:10078000882309F0D6C080911201882309F0D1C0D6
:1007900080911301882309F0CCC0CB3108F4BAC092
:1007A00080911601882309F0B5C080916C008823E0
:1007B00009F0B0C0C0911701CC2309F0ABC08D2D5A
:1007C000A9DD882309F4B5C0153009F0B2C08091C5
:1007D0003201843008F4ADC080914D0190914E01FA
:1007E0008558934008F4A5C0C09369008091240106
:1007F000A82EBB24E1E0EE2EF12C60913B01CCE46D
:10080000D0E020E030E073E0A3E3B1E08D01C5016A
:10081000022E02C0959587950A94E2F7AC014170CB
:10082000507080FD2CC0FE018491E82FFF27E45E0C
:10083000FE4F8081981648F0C701022E02C0880F33
:10084000991F0A94E2F7682B0CC0C701022E02C060
:10085000880F991F0A94E2F780956823F801408376
:1008600051838D919C911197885E934040F0C70110
:10087000022E02C0880F991F0A94E2F7C82A71500D
:100880002F5F3F4F0E5F1F4F1296219677FFBFCF0E
:1008900060933B0124E0D21619F048E0D41651F4DD
:1008A0008091570181FF06C0EC2DFF27E45DFF4FCB
:1008B000849105C0EC2DFF27E45CFF4F8491809369
:1008C000240120910B012778309124018C2D832B5A
:1008D000992773E0880F991F7A95E1F7282B2093C9
:1008E0000B012091FA00237C832F9927880F991FF1
:1008F000880F991F282B2093FA002091F900237C60
:100900008C2D9927880F991F880F991F282B2093CA
:10091000F9000FC080910B01877880930B018091C3
:10092000FA00837C8093FA008091F900837C8093A5
:10093000F900809131018F5F80933101883010F090
:100940001092310134DDDF91CF911F910F91FF9013
:10095000EF90DF90CF90BF90AF909F900895CF938E
:1009600080910E01882321F0809146018B3031F077
:1009700010920E0110920D0110920C0120911B019A
:100980002223B1F485B394E0892785BB809151017E
:1009900090915201885E934040F08CB58093F400B2
:1009A0002CBD109252011092510181E080931B01E5
:1009B000D1DB1FDCFBDD80911901882321F0A99890
:1009C00035DC10921901809146018F3151F48091EC
:1009D0006800882331F02ADC809168008150809380
:1009E000680080915001209146019091F90082FFAA
:1009F00002C0916001C09E7F9093F9002F31A1F059
:100A0000839B12C080916C00882371F49091140133
:100A1000992351F480911F018A3120F481E0809361
:100A20006A0002C090936A00839B04C0B09906C01C
:100A3000989904C08091FA00826003C08091FA0006
:100A40008D7F8093FA0080911801882329F080918E
:100A5000F90080688093F900809146015BDC88236F
:100A6000D9F080912101893E48F08091F90082609F
:100A70008093F90081E08093160111DB80911401CD
:100A8000882351F080911501882309F408DB8091B7
:100A9000FA008C638093FA0020916C00222391F479
:100AA00080911F018D3170F080915301909154011C
:100AB000C39740F0839B06C081E080930F01209391
:100AC000100102C010920F01829904C081E080934E
:100AD0006C0002C010926C0080916C00882321F49D
:100AE00080916A00882321F08091F900806403C01E
:100AF0008091F9008F7B8093F900809146018B50A3
:100B0000823060F4809121019091F900893E10F0CB
:100B1000926001C09D7F9093F900E9DA9091E8001E
:100B2000913039F48091E700882319F49093E7001D
:100B30001FD6C0914601CF3109F4E4C08091110164
:100B40008823D1F08C2FE6DB282F882339F480917D
:100B5000550190915601855F914050F4222309F48C
:100B6000D1C080915501909156010B9708F4CAC0ED
:100B7000969A10921101C6C080911501882309F43C
:100B800056C08C2FC7DB882379F0809101018093B8
:100B90004701809102018093480180910301809375
:100BA0004901809104010AC0809347018093480164
:100BB00080910501809349018091060180934A014B
:100BC00090911F019B3020F480911701882341F4FC
:100BD000973208F097C080911701882309F092C0DE
:100BE0001092150180911601882309F08BC0809125
:100BF0001401882309F086C080916B00882309F0D6
:100C000081C080910E01882361F0CB3051F4809136
:100C10000D01882331F0B09B02C0A898C098A89A13
:100C200071C0989B02C0A898C098C09A6BC0809170
:100C300057019927807C907080389105F9F443988A
:100C40008C2F68DB882379F0809101018093470124
:100C500080910201809348018091030180934901B2
:100C6000809104014DC08093470180934801809199
:100C70000501809349018091060142C0809157018E
:100C80009927807C9070803C9105C9F443988C2F03
:100C900041DB882379F08091FB00809347018091AC
:100CA000FC00809348018091FD0080934901809170
:100CB000FE0026C080934701809348011BC08C2F03
:100CC00029DB882399F080911F018B3128F0839BC9
:100CD00003C0439A449A01C0439810924A0110926B
:100CE000490110924801109247010CC080934801BD
:100CF000809347018091FF0080934901809100011A
:100D000080934A01809146018F31A9F480911F019F
:100D10008B3088F41092150180911601882359F4C4
:100D200080911401882339F480910E01989B02C0B0
:100D3000A898C098C09AF6DA13CECFE5D4E0DEBF0B
:100D4000CDBF88E285BB85E088BB969A94988FE2F8
:100D500084BB87BB82E581BB84E58DB91EB883E483
:100D600088B98EE886B986E087B98AB780688ABF75
:100D700080E88BBF8AE085BF92D9FDD09DD9A8D9E4
:100D8000789480E038D580914201882389F481E00D
:100D900032D580914201882341F482E02CD582E053
:100DA0008093E80081E0E4D403C081E08093E80010
:100DB000D6DD80E090E0ACC71F920F920FB60F9285
:100DC00011242F933F934F935F936F937F938F9350
:100DD0009F93AF93BF93CF93DF93EF93FF9387ECF2
:100DE00082BF80911B01882311F010921B0180911A
:100DF00051019091520101969093520180935101BB
:100E000080911101882349F08091550190915601FC
:100E100001969093560180935501839B0DC080915C
:100E20006900882349F080914D0190914E0101960F
:100E300090934E0180934D0180911F018D3168F098
:100E400080911001882349F08091530190915401C1
:100E50000196909354018093530180913B01C82FD8
:100E6000DD2740E050E063E0E3E3F1E0CE01042E53
:100E700002C0959587950A94E2F780FF0EC0DF01C6
:100E80002081318180819181895E934018F4C9016C
:100E9000019601C0C9018D939C9361504F5F5F4FD4
:100EA000329667FFE3CFFF91EF91DF91CF91BF9132
:100EB000AF919F918F917F916F915F914F913F91F2
:100EC0002F910F900FBE0F901F9018951F920F92A9
:100ED0000FB60F9211242F933F934F935F936F930D
:100EE0007F938F939F93AF93BF93EF93FF9381E093
:100EF00080931701D4D8FF91EF91BF91AF919F914B
:100F00008F917F916F915F914F913F912F910F90B2
:100F10000FBE0F901F9018951F920F920FB60F9251
:100F200011248F9380911501882381F480911401FD
:100F3000882361F480911601882341F48091170180
:100F4000882321F481E08093180143988F910F90BA
:100F50000FBE0F901F9018951F920F920FB60F9211
:100F600011248F9381E080931A018F910F900FBE0F
:100F70000F901F90189510BC8BE089B91BB888E9B9
:100F80008AB986E880BD86E085BD0895982F2FB781
:100F90002078F8948091D200E82FFF27E359FF4F83
:100FA00090838091D2008F5F8093D2008091D20095
:100FB000843610F01092D2008FB7822B8FBF089525
:100FC000DF92EF92FF920F931F93CF93DF93982FAF
:100FD000F62EE42ED22E80915801882339F1C92FA4
:100FE000DD27892FD3DFCF0DD11D8F2DCFDFCE0D84
:100FF000D11D8E2DCBDFCD0DD11D8D2DC7DFDD2079
:1010000051F078011D2DF70181917F01C80FD11D8D
:10101000BDDF1150C1F7D095C195DF4F8D2F9927B6
:10102000B5DF8C2FB3DF5498949A559ADF91CF9106
:101030001F910F91FF90EF90DF9008951F920F92F4
:101040000FB60F9211248F939F93EF93FF9380918C
:10105000D100E82FFF27E359FF4F80818CB98091A1
:10106000D1008F5F8093D1008091D100843610F041
:101070001092D1009091D1008091D200981749F43C
:1010800055985E9A569A1092D2008091D200809321
:10109000D100FF91EF919F918F910F900FBE0F9014
:1010A0001F901895282F30E0809146018B3059F41D
:1010B00023FF09C080910E01882309F431E081E00B
:1010C00080930E0106C080910E01811131E01092D3
:1010D0000E0190910E01992381F080910D0124FF62
:1010E00007C0882309F431E081E080930D0108C036
:1010F000811131E010920D0103C090930D011BC0CE
:101100009923C9F080910C0125FF0BC0882309F4B5
:1011100031E081E080930C01809312011092130161
:101120000CC0811131E010920C0181E08093130119
:101130001092120102C090930C0131111CD9089534
:101140000895EF92FF920F931F93CF93DF93CDB744
:10115000DEB72B970FB6F894DEBF0FBECDBF7C0174
:10116000FC01818199278031910509F47AC0813190
:10117000910534F58430910509F448C08530910516
:1011800064F48230910509F449C0833091050CF074
:101190004CC0892B09F40FC130C18730910509F487
:1011A00078C08830910524F4069709F44CC025C115
:1011B0008830910509F485C0099709F4F2C01DC172
:1011C0008531910509F449C08631910574F4823165
:1011D000910509F43EC0823191050CF44EC0833173
:1011E0009105C9F1449799F108C18731910509F436
:1011F00078C0873191050CF480C08838910509F4D6
:10120000DFC08938910509F0F8C0D5C0F7018381A6
:10121000809357018091570145DFCDC0F70183814D
:1012200080935701809157013DDF0DEE10E02EE0D5
:1012300043E060914601F7018281C2DE8091450161
:1012400080935001DAC081E080931901D6C093D811
:10125000D4C080E803C080EC01C080E480935701D3
:10126000CCC0809146018350843018F481E0809393
:10127000140181E080931201C0C080914601875023
:10128000843018F481E08093140181E0809313018D
:10129000B4C01092E6008091E60088608093E6007A
:1012A000F70183818093590184818093570185815F
:1012B00080935A0100E010E020E041E06091460197
:1012C0009AC0F701838180935901848180935701EB
:1012D000858180935A016BD809EE10E024E048E044
:1012E00087C0F701838180935901148160D8E12F71
:1012F000FF27EC5AFF4F849144C0F701838180930C
:1013000059011481212F332720FF02C082E001C040
:1013100080E090915901981738F1143028F59430F5
:1013200018F5F901EC5AFF4F8491A82FBB27492FDC
:101330005527A550BF4FA40FB51FF70185818C938A
:1013400021FF12C0923080F081E08127E82FFF2733
:10135000EC5AFF4F8491A82FBB27A550BF4FA40F75
:10136000B51FF70185818C9382E08093E80081E0CE
:10137000FFD11092E7001BD8E12FFF27EC5AFF4F57
:101380008491E82FFF2780915901E550FF4FE80F26
:10139000F11D80818093EA0009EE10E024E047E12E
:1013A00027C082E08093E80081E0E2D11092E7005C
:1013B00080E28093E60000E010E020E041E018C009
:1013C000F7018381948189839A8385818B83893016
:1013D00010F088E08B838B819927AC0169817A8139
:1013E000CE010496A0D18E010F5F1F4F2BE048E87D
:1013F00060914601F7018281E3DD2B960FB6F894E8
:10140000DEBF0FBECDBFDF91CF911F910F91FF9037
:10141000EF90089584B5885B83BD88B7806888BFE6
:1014200089B7806889BF089589B78F7789BF88B7E2
:10143000806888BF08951F920F920FB60F921124F3
:101440002F933F934F935F936F937F938F939F93CC
:10145000AF93BF93CF93EF93FF938BB199278C7189
:101460009070892B99F05F9BC5C08BB199278C71C7
:101470009070892B09F4BEC0CCB15F9BBBC08BB10F
:1014800099278C719070892BB9F7B4C0C3DF409154
:101490003C01842F99278F70907082309105A1F1C3
:1014A000833091052CF4009771F00197F9F08BC00F
:1014B0008430910509F456C0843091059CF105975C
:1014C00009F46EC080C0CCB18C2F992790933F0156
:1014D00080933E0180914601C81711F0CC23D1F5CD
:1014E000406840933C01C093580134C0CCB1809116
:1014F0003E0190913F018C0F911D90933F0180938D
:101500003E01C093D5005BC0CCB180913E0190916B
:101510003F018C0F911D90933F0180933E01C0933A
:10152000D4004DC0CCB1C093D300CC23C9F01092ED
:101530003D0180913E0190913F018C0F911D909350
:101540003F0180933E0147FF05C0CB3018F04F7735
:1015500040933C0180913C018F5F80933C014AC0E5
:101560004E5F2EC0CCB180913E0190913F018C0F17
:10157000911D90933F0180933E0147FF07C08091EA
:101580003D01E82FFF27ED52FF4FC38380913D01BE
:101590008F5F80933D019091D300891758F10FC060
:1015A000CCB18C2F9927382F222780913E01909122
:1015B0003F01820F931F90933F0180933E014F5F45
:1015C00040933C0117C0CCB12FDF80913E01909138
:1015D0003F018C0F911D90933F0180933E01892B19
:1015E00039F480913C0187FF03C083ED90E0A9DDD1
:1015F00010923C01FF91EF91CF91BF91AF919F91DC
:101600008F917F916F915F914F913F912F910F90AB
:101610000FBE0F901F9018951F920F920FB60F924A
:101620001124559902C09498549A56980F900FBE61
:101630000F901F9018951F920F920FB60F921124C2
:101640002F933F934F935F936F937F938F939F93CA
:10165000AF93BF93EF93FF9310923C01E5DEFF91B0
:10166000EF91BF91AF919F918F917F916F915F911A
:101670004F913F912F910F900FBE0F901F90189593
:10168000AF92BF92CF92DF92EF92FF920F931F9390
:10169000CF93DF937C015B01EA01DD24CD2C0FB6F3
:1016A00007FE03C091E0C92EF89400E411E0809198
:1016B000400190914101892B49F0D801ED91FC91B5
:1016C0008F010C5F1F4F84819581F5CFCE01069667
:1016D00068D1FC010097B9F0D8018D939C93E0820A
:1016E000F182C283D38314821582209749F0DC01F2
:1016F0001696F501AE0181918D9341505040D9F776
:10170000E39A81E0D82ECC2009F078948D2D99278A
:10171000DF91CF911F910F91FF90EF90DF90CF90CD
:10172000BF90AF900895A0E02A2F0FB607FE02C029
:1017300021E0F894E399A1E0E398222309F078945A
:1017400020E030E02417350778F4FC01E199FECF62
:101750007FBB6EBBE09A8DB381932F5F3F4F6F5F6E
:101760007F4F2417350790F3A111E39A0895089548
:10177000682F10927201109271018BEF90E090939C
:101780005E0180935D01FC014FE050E0819120916A
:10179000710130917201280F311D30937201209335
:1017A00071014150504057FFF1CF309370012093A9
:1017B0006F01EFE5F1E0ABEFB0E08D91819381E057
:1017C000EE36F807D1F3CCF3862F9927009719F05E
:1017D000019741F0089542E150E06FE571E080E04B
:1017E00090E006C042E150E06FE571E082E190E0F8
:1017F00047DF089508951F93CF93C82F10E00FB6C9
:1018000007FE02C011E0F8948C2F992781309105D2
:1018100071F0823091051CF4892B21F017C00297DA
:1018200071F014C042E150E060E070E004C042E1B9
:1018300050E062E170E08FE591E075DF07C048E0BD
:1018400050E068E570E08BEF90E0A1D1C23098F5F0
:10185000EBEFF0E0AFE5B1E09F018D91819381E086
:10186000EA30F807D1F3CCF31092720110927101B3
:1018700030935E0120935D01F9014FE050E08191CA
:101880002091710130917201280F311D3093720146
:10189000209371014150504057FFF1CF80916F016B
:1018A000909170018217930721F481E080934201A7
:1018B00002C010924201112309F07894CF911F9138
:1018C00008951F920F920FB60F9211242F933F93FA
:1018D0004F935F936F937F938F939F93AF93BF9338
:1018E000EF93FF93A0914001B0914101109709F44B
:1018F00046C08D919C9111972091430130914401F4
:10190000820F931F9FBB8EBB8CB3992796958795AB
:10191000AC014170507080FDF7CFE09A8DB3FD01AE
:10192000E20FF31F9681891719F09DBBE29AE19AA5
:101930002F5F3F4F3093440120934301FD0182818B
:10194000938128173907E0F08481958190934101B4
:10195000809340015093440140934301CD01BBD09B
:101960008091E800882329F08091E80081508093DD
:10197000E8008091400190914101892B09F4E3989E
:10198000FF91EF91BF91AF919F918F917F916F9157
:101990005F914F913F912F910F900FBE0F901F902D
:1019A0001895CF93DF93AC01029710F442E050E01A
:1019B00020E030E0A0917501B0917601BD01F90100
:1019C000109709F44CC08D919C911197841795073D
:1019D00031F14817590738F42115310519F08217EC
:1019E000930708F49C01FD01A281B381109759F778
:1019F00021153105A1F1C901841B950B049708F449
:101A0000A901DB01E0E0F0E0109749F18D919C9194
:101A1000119782179307F9F44217530779F4ED01F0
:101A20002A813B81CD010296309719F022833383BE
:101A30004FC030937601209375014AC0241B350BAB
:101A4000FD01E20FF31F41935193225030402D933B
:101A50003C93CF013DC0FD01A281B381D5CF8091E0
:101A6000730190917401892B41F48091E20090916F
:101A7000E3009093740180937301E091E000F09192
:101A8000E100309741F4EDB7FEB78091E40090910A
:101A9000E500E81BF90BA0917301B09174019F015F
:101AA0002A1B3B0B2417350788F0CA01029628171A
:101AB000390760F0CD01840F951F02969093740151
:101AC000809373014D935D93CD0102C080E090E05F
:101AD000DF91CF910895CF93DF93009709F454C01D
:101AE000DC011297ED011A821B82809175019091A1
:101AF0007601009721F1FC0140E050E0EA17FB0776
:101B000018F1ED01EA83FB832D913C911197C20FEF
:101B1000D31FCE0102968E179F0771F48A819B8195
:101B2000280F391F2E5F3F4F2D933C9311978281D1
:101B30009381FD01828393834115510559F4B0933C
:101B40007601A093750120C0AF010280F381E02DE2
:101B50003097A1F6EA01AA83BB83CA0102962881C5
:101B60003981820F931F8A179B0771F48D919C9185
:101B70001197280F391F2E5F3F4F28833983FD01AE
:101B8000828193818A839B83DF91CF910895FB01AA
:101B9000DC0102C005900D9241505040D8F70895E5
:101BA00097FB4ED09F3738F0FEE9F91B982F872F0F
:101BB000762F6B2F05C052C09695879577956795C0
:101BC000F150D0F73EF490958095709561957F4FD8
:101BD0008F4F9F4F0895E89403C097FB0EF4F3DFF7
:101BE000B62F672F782F892F9EE9002405C09A957C
:101BF000BB0F661F771F881F11249923A1F088232C
:101C0000B2F79F3F59F0BB0F48F421F4002011F4C4
:101C100060FF04C06F5F7F4F8F4F9F4F881F979566
:101C2000879597F908951AC0052E092607FA440FDB
:101C3000551F5F3F79F0AA27A51708F051E0479597
:101C4000880F991F9F3F31F0BB27B91708F091E02B
:101C5000879508959F919F91112457C066277727F4
:101C6000882799270895592F482F372F262FDCDFF3
:101C700001D0C2CF992339F0552329F09F575F57E0
:101C8000950F13F4CAF1EDCF91589F3FE1F3A62FC2
:101C900000241124BB2766275527F8E0A69520F4D9
:101CA000020E131EB41F651F220F331F441F551F42
:101CB000FA95A1F7F8E0E72F7727F8E0E69520F40A
:101CC000130EB41F651F7A1F330F441F551FAA1F21
:101CD000FA95A1F7F82F8827F69520F4B40F651F21
:101CE0007A1F8E1F440F551FAA1FEE1FFF23A1F757
:101CF00088231AF4939539F408C0000C111CBB1FFB
:101D0000661F771F881F012808959FEF80EC0895B4
:021D1000FFCF03
:101D1200030400010205070803010101010000009C
:101D220000000000000000000000000000000000B1
:101D320000000000000000000000000000000000A1
:101D42000000000000000000000000000000000091
:101D52000000000000000000000000000000000081
:101D62000000000000000000000000000000000071
:101D72000000000000000000000000000000000061
:101D82000000000000000000000000000000000051
:061D9200000077012000B3
:00000001FF
